:1000000000308A00C3290000FF00030E8301A10015
:100010007F08A0000A08A8008A01A00E0408A20018
:100020007708A3007808A4007908A5007A08A6003C
:100030007B08A700831383128C308400801D222844
:100040008C193528220884002308F7002408F800BA
:100050002508F9002608FA002708FB0028088A006E
:10006000210E8300FF0E7F0E09008A1137286808D1
:1000700093008C118A112228713084000008031922
:1000800051280130F800BF30F7006400F70B452815
:10009000F80B43284230F700F70B4C286400800B24
:1000A00041280034831605178312051F59280513AC
:1000B0005A2805178316051383128A11632AF10142
:1000C0007108F93C031C81287018682805136928F9
:1000D0000517831605130130F00670187328831274
:1000E000851375288316831285178316851364007C
:1000F0001F30F700F70B7A2800000000F10A831286
:10010000602883160513831205178316851383123F
:1001100085178A11B12A6908840072088000840A50
:100120008001E90A00347308F801720203189B2861
:100130007208F700A728F7010830F400F20DF70D58
:10014000730877020318F700F80DF40B9E280034AB
:1001500078087008F2006430F30093207708F0000C
:1001600078083030031DBB28F11CC228F119C228C1
:10017000711A2030BE28F11171127114F807780835
:10018000F2008B207008F2000A30F3009320770809
:10019000F00078083030031DD328F119D728711CDE
:1001A000D728711A2030F8077808F2008B203030F9
:1001B000F0077008F2008B200034BC01391CE228E3
:1001C0003910E32839140034391C1029831686129B
:1001D0008312861264004730F700F70BED28000009
:1001E000831686128312861664004730F700F70BD9
:1001F000F7280000831686128312861264004730A7
:10020000F700F70B01290000831686128312861669
:1002100064001830F700F70B0B29000000002329B9
:10022000831686128312861264008530F700F70B5E
:100230001729831686128312861664006F30F70022
:10024000F70B202900000034F3017308073C031C5E
:100250006C2972080139F400BE08031931290030F5
:1002600032290130F500BD08031938290030392939
:1002700001307505003A03194C297408F500031084
:10028000BB0CBA0C030801397506013C031D4C294F
:100290008430BB060830BA06F408031D5129DD205E
:1002A0006729BD080319BC0ABD0803195929003084
:1002B0005A290130F5003C08053C0319612900303A
:1002C00062290130750503196729E420DD20E42047
:1002D0000310F20CF30A252900343910FF30BB005B
:1002E000BA00BC010130BD00BE01BF013F08093C9E
:1002F000031C7F297E30F2002421BF0A7629BD012C
:10030000BF013F080F3C031C8E2929303F078400A2
:100310000008F100F2002421BF0A8129BF01700802
:100320008400000803199D29700884000008F1006A
:10033000F2002421F00ABF0A8F290130BE00FF30ED
:10034000BA06BB063A08F20024213B08F200242139
:10035000BE010130BD007E30F20024218A11FD2A49
:100360001230F202031CC22972308400FC30800576
:100370000310800C800C00080319C229C0296400F6
:10038000800BBF29003484011F30830583161F12A0
:100390009F121B0880399B0007309C00823083121B
:1003A000A9009830AA00AB004030AC00AD00AE0010
:1003B0006030AF008630B000B430B1006030B200C1
:1003C000A430B300B400B5006130B6000330B7000C
:1003D000F030B800E90183160108C03981000E3001
:1003E000F700073083128101813084000008F03962
:1003F0000738800064000008F739F719F0397704EE
:100400008000900183161F129F121B088039D33879
:100410009B001F1383121F179F1783169F138312AE
:100420001F149412831606118614061200308312CC
:1004300094008316940007309C0005086400023085
:10044000F700F70B212A00001C0883120D138316F6
:100450009D018611831286118316061183120611DF
:1004600083168610831286108316851383128517D0
:1004700083160513831205172030F8001F08C739AB
:1004800078049F00950183168611831286110C3023
:1004900097000030F8000438920064308316920010
:1004A00062308F00023083129500EA0183168610B5
:1004B000831286106430F1003C206A08EA0A043C8A
:1004C000031D642A5228EA018316861083128614BB
:1004D0000130F1003C201F151F196C2A1E085F3CDB
:1004E000031C562A83168610831286100030F800EB
:1004F0001F08C73978049F0064001F30F700F70B0E
:100500007F2A000000001F151F19842A1E08F7000B
:10051000F70CF70C3F30F7057708283EEB00083062
:10052000F8001F08C73978049F0064001F30F700E7
:10053000F70B982A000000001F151F199D2A1E0C9A
:10054000EC00EC0CEC0C1F30EC0595010030F800D1
:10055000043892006B0883169200133083129500C2
:100560005F280230F000FA30F1003C20F00BB32A93
:1005700083168610831286142030F8001F08C739AE
:1005800078049F0064000F30F700F70BC52A0000C5
:100590001F151F19C92A1E08ED0083168610831225
:1005A00086104030E9007030F2008B203D30F200C0
:1005B0008B206B08F0001B30F100A8202030F200E7
:1005C0008B207230F2008B203D30F2008B206C08C3
:1005D000F0001B30F100A8202030F2008B20753095
:1005E000F2008B203D30F2008B206D08F0001B30B4
:1005F000F100A8204030F0006D293830F000FA30CA
:10060000F1003C20F00BFF2AEF010130EE006F08F3
:10061000033C031C332B031D112B6E08E83C031C09
:10062000332BEA016A086C02031C2F2B8316061178
:10063000831206156E08F200B0218316061183128C
:1006400006116E08E83CF0000330F1006F08031C4F
:100650006F0FF1027008F200B021EA0A122BEE0AC5
:100660000319EF0A072B83160611831206150A30A9
:10067000F0008230F1003C20F00B392B831606117C
:0806800083120611422B6300F6
:04400E003827FC3F14
:00000001FF
